:0600000002005B0236D194
:03000B0002330EAF
:030013000233179E
:03001B0002002BB5
:030023000235851E
:10002B0032416C636F726E204D634272696465205E
:10003B00496E632E20536372697074204F53202DC9
:10004B002056657273696F6E20362E353320202053
:10005B00C2AF75D0007581567A00122D8975B81014
:10006B0075A813787FE4F6D8FD758DFD758BFD753E
:10007B008C88758A0875892175880475368875355D
:10008B00087598C07E007F409020007400F0A3DEBE
:10009B00FCDFFA75A0887800E2F52C75A088780251
:1000AB00E2F52DD2AFD28CD28E12213590000012F8
:1000BB0032D1FAA31232D1FBA31232D1FCA31232EA
:1000CB00D1B4600040027460FD4C6018A31232D1B1
:1000DB00F540A31232D1A31232D1F54E9000021289
:1000EB00210D6017903A25122D037537287455F59D
:1000FB0099780000D8FDD20302019974AAF599787A
:10010B000000D8FDC203903A36122D03122CC17594
:10011B00382890000F1232D1A2E792091230EA75FB
:10012B004520754400754B00754A30854E4FE54EA2
:10013B006056900020A3A3D54FFB75A02E780085A9
:10014B004E4F1232D1F2A3081232D1F2A308B800EB
:10015B000205A0D54FEC854E4F8545828544831211
:10016B0013A6A3A31232D1540F854B82854A83F079
:10017B00A385824B85834A854582854483A3A385CA
:10018B008245858344D54FD112318D1230907A0040
:10019B00122D89D29C1201C21202193001F7C20131
:1001AB002003F2122FB6120C31120F7412110B1214
:1001BB0013C81213CE80DE75D0089021007F5A7EB3
:1001CB0003E0F5F0A3E0F8A3E0F9686034E5F05440
:1001DB007FB400051202538028B401051204EB8092
:1001EB0020B402051202B08018B40505120A7F80F4
:1001FB0010B40905120B7E8008B4080512057F8028
:10020B0000E5822406F5820FDEB775D00022300799
:10021B0036E4B530130530122CC1903A97122D03EA
:10022B00903AC0122D15801F7405B5301005309013
:10023B003AE9122D03903B12122D15800A745FB50B
:10024B0030050530122CE122AC83AD828F8389827D
:10025B0075D00075A0247800E0FB75F000E425F064
:10026B00F5F00582E5826508602DE0F208DBEF050D
:10027B0082C5F003547FB5F01E858209902400E0FF
:10028B00FBA3D20A753803121419300B03122FB6C5
:10029B0075D0088982800675373C75D008E5828C4D
:1002AB00838D82F02285820C85830DE50FC3945AD2
:1002BB0023245BF50B850F83850982E030E70FB4B0
:1002CB00F8005007850B82758325F00204D1850B4E
:1002DB0082758325E0B49000400EB4A0004053B467
:1002EB00F0030203890204D1540FB540F8E5090469
:1002FB00B508030204E4850F83F582E030E70302BF
:10030B0004D11582E00509C3943CB4080050209039
:10031B002400F5F0E540F0A37403F0A3E5F0F075CD
:10032B00D0007BFF902400D20A12141975D008025A
:10033B0004D1540FB540AEE50904B508030204E43B
:10034B00850F83F582E030E7030204D160B4158298
:10035B00E00509C3943CB408005020902400F5F04C
:10036B00E540F0A37402F0A3E5F0F075D0007BFF3D
:10037B00902400D20A12141975D0080204D1E50892
:10038B00C39509B4070050030204B8850F83850990
:10039B0082E0B47F4A0582E0B47F028003B5403F20
:1003AB000582E0B402390582E0B47F028008B41004
:1003BB00028003B430290582E0B40703020470B451
:1003CB00010DE508C39509B4090050690204B8B4DE
:1003DB00060DE508C39509B40A0050060204B802DD
:1003EB0004A30582E020E7F760F5B4210050F0F597
:1003FB000B0582E020E7E80582E020E7E2F5F00557
:10040B0082E020E7DA03548045F0F5F0858209900D
:10041B002400E540F0A37428F0A3E50B14F0A3E54A
:10042B00F0F075D0007BFF902400D20A12141975DE
:10043B00D0080204D10582E020E75DC3943075F04B
:10044B000AA4F5F00582E020E74EC3943025F07541
:10045B00F00AA4F5F00582E020E73DC3943025F0C7
:10046B0014F5F080090582E020E72DC3F5F0058235
:10047B00E0B4F724858209902400E540F0A37418BA
:10048B00F0A3E5F0F075D0007BFF902400D20A12A8
:10049B00141975D0080204D130E7030204CC753768
:1004AB003C850B8275832574F7F00204D1850F838D
:1004BB00850982E020E70A0582E582B508F502048A
:1004CB00E48582091509850C82850D83E50904F005
:1004DB00F509650860030202C0850C82850D832235
:1004EB00AC83AD8275D010E508B5090302057485A0
:1004FB000F83850982E00509B4F5ECA8091509E518
:10050B0008C398B405005003020574120A28B540BD
:10051B0045902400F0A3F5F0120A28FBB403005019
:10052B003525F0F5F0120A28602CB440005027F95D
:10053B0025F0F5F0E92405FAE508C39509FEB51297
:10054B00004026120A28F0A325F0F5F0D9F5120A7F
:10055B0028B5F002800875373C05090204F275389E
:10056B0003120A3888090204F275D008E5098C8356
:10057B008D82F022AC83AD8275D010E508B50903EE
:10058B00020648850F83850982E0B4F102800405D9
:10059B000980E88509F005F0E508B5F00875D00885
:1005AB008C838D8222850F8385F082E0B4F10280EB
:1005BB00DEB4F202800405F080DEE508B509030223
:1005CB000648850F83850982E00509B4F10F740194
:1005DB001209DE75A02078C8E4F20205C5B4F21644
:1005EB00120A0530E00AC2E0C2E11209DE0206532C
:1005FB0075373C0205C5F5F0120A0520E006753784
:10060B003C0205C5F8E5F0B4F009E8D2E11209DEC9
:10061B000205C5E830E10BC2E11209DEE5F024F07A
:10062B00F5F075A02078C8E275A033780028F8E5BE
:10063B00F0F2E80475A02078C8F20205C575D00861
:10064B00E5098C838D82F02275A02078C8E2B40373
:10065B0000500675373C0206F175A033780028F878
:10066B0018E2F5F0790018E229F918B8FFF9E9B5A5
:10067B00F002800675373C0206F175A033780090C6
:10068B0020C412098912091EB4000675373C0206F4
:10069B00F1B40121E49020B4F0A3F0A3F0A3F09007
:1006AB0020B8F0A3F0A3F0A3F09020BCF0A3F0A32C
:1006BB00F0A3F080129020B41209899020B812098F
:1006CB00899020BC1209897900C0129020C8E0FAE9
:1006DB001AE4F5F0E2F3080905F0EAB510F6E5F0D7
:1006EB00F0D0120206F402064812091EB402399029
:1006FB0020B4E0B4FF1AA3E0B4FF15A3E0B4FF10DD
:10070B00A3E0B4FF0B120A05D2E31209DE02073392
:10071B007582B4E0700FA3E0700BA3E07007A3E049
:10072B00B5400280030207FC75A03378009020C00F
:10073B001209899020C0E0A3B40016E0A3B4001105
:10074B00E0A3B4000CE0B404028009B4003B020740
:10075B00F90207F9E2B4003108E22403FEE2FE08D5
:10076B00902400E540F0A3E2F008A3EEB510F8905A
:10077B00240075D000D20A75380312141975D010E5
:10078B00120A0530E3090207FC75373C0207F975BD
:10079B00A02078C412094612091EB4021475A020B9
:1007AB0078B812094675A02078B41209467405F082
:1007BB00A3E4F0A37401F0A375A02078C8E2F97547
:1007CB00A0337800E2F008A3E8B511F875A02478FF
:1007DB000075F000A982E20825F0F5F0E8B511F6F6
:1007EB00E5F0F0A3E50FC3945AFA091208BC02080E
:1007FB00659020BCE0700EA3E0700AA3E07006A326
:10080B00E07002805514F0B4FF187582BEE014F04E
:10081B00B4FF0F7582BDE014F0B4FF067582BCE027
:10082B0014F0E50FC3945AF5F0902100E5822408EB
:10083B00F5827A01E0547FB40816E5F0B512028018
:10084B000FAD82AE83AFF01208688D828E838FF06E
:10085B00E5822408F5820ABA03DA0206F190240035
:10086B0075A02078C412094675A02078B4120946E9
:10087B0075A02078B812094675A02078BC120946DD
:10088B0075A02078C8E2F975A0337800E2F008A3D0
:10089B00E8B511F875A024780075F000A982E2087C
:1008AB0025F0F5F0E8B511F6E5F0F0A3091208BC58
:1008BB002290340074F1F0A375A0247800E208B400
:1008CB00F007F0A3E4F0A3801CB4F10A74F0F0A3DA
:1008DB007401F0A3800FB4F20A74F0F0A37402F069
:1008EB00A38002F0A3E8B511D474F2F0A3A982900F
:1008FB00240075A0347800E2F008A3E582B511F767
:10090B0075D000902400AB11AA12D20A122D937548
:10091B00D01022C082C0839020C4E0B40016A3E0A4
:10092B00B40011A3E0B4000CA3E0B401028007B43F
:10093B00020280027400D083D08222E20860167417
:10094B00FDF0A30808E218F0A3E218F0A3E218F0F8
:10095B00A3E2F0A322E208601174FEF0A308E218F0
:10096B00F0A3E218F0A3E2F0A322E208600C74FFFC
:10097B00F0A3E218F0A3E2F0A322E2F0A322C0114D
:10098B00E2F9B9FD1708080808E218F0A3E218F01D
:10099B00A3E218F0A3E2F00808088033B9FE14E4D0
:1009AB00F0A3080808E218F0A3E218F0A3E2F0089D
:1009BB0008801CB9FF10E4F0A3F0A30808E218F0BC
:1009CB00A3E2F0088009E4F0A3F0A3F0A3E2F0089F
:1009DB00D01122C009C082C083C0E0E50FC3945A76
:1009EB00F509902100E5822408D509FB2407F5823F
:1009FB00D0E0F0D083D082D00922C009C082C0835E
:100A0B00E50FC3945AF509902100E5822408D50916
:100A1B00FB2407F582E0D083D082D00922C083C0AB
:100A2B0082850F838882E008D082D0832275D00024
:100A3B007BFF902400D20A121419E513B400028034
:100A4B002FB40214E50FC3945AFA850F83850982DC
:100A5B00E516FBD20A122D93E50FC3945AFA74AA2A
:100A6B003012027455902400F07B01D20A122D93A0
:100A7B0075D01022AC83AD8275D010A809E508C3E0
:100A8B0098B40C005003020B73850F83E509240205
:100A9B00F582E0B43A028066B42D60A809E508C37C
:100AAB0098B417005003020B73E5092416F582E086
:100ABB00B40D48902400A8097919120BD4120C0418
:100ACB0008791A120BD4120C0408791B120BD412CE
:100ADB000C04E82406F8791C120BD4120C040879C8
:100AEB001D120BD4120C0408791E120BD4120C0419
:100AFB00791FE4120C04E8F5098080020B6EE509FE
:100B0B00240BF582E0B40D5BA809E8F9120BD4B401
:100B1B001800504C120A28B43A46120BD4B43C00BD
:100B2B00503E120A28B43A38120BD4B43C00503061
:100B3B00753803902400E9F8791C120BD4120C04BD
:100B4B0008791D120BD4120C0408791E120BD41247
:100B5B000C04791FE4120C04E509240CF5094186F9
:100B6B0075373C0509020A8675D008E5098C838D1B
:100B7B0082F022AC83AD8275D010A809E508C3982A
:100B8B00B405004039850F83850982E0B4432AA858
:100B9B0009E5092403F8E8120BD4601AB46300507A
:100BAB001514758330F582E0D2E2F0753803E50950
:100BBB002405F50980C475373C0509020B8575D0F2
:100BCB0008E5098C838D82F022C083C082850F8358
:100BDB008882E0080582C39430B40600501475F087
:100BEB000AA4F5F0E008C39430B40A00500425F0D1
:100BFB00800274FFD082D08322C0F0F5F0E540F084
:100C0B00A37428F0A3E9F0A3E5F0F0A324282903AB
:100C1B00547FF075D0007BFF902400D20A12141978
:100C2B0075D010D0F022908800E0F8C52C6830E029
:100C3B000CC0E0A26075F000120D2AD0E030E10C80
:100C4B00C0E0A26175F001120D2AD0E030E20CC0B9
:100C5B00E0A26275F002120D2AD0E030E30CC0E086
:100C6B00A26375F003120D2AD0E030E40CC0E0A2B1
:100C7B006475F004120D2AD0E030E50CC0E0A265DB
:100C8B0075F005120D2AD0E030E60CC0E0A26675B7
:100C9B00F006120D2AD0E030E708A26775F00712B4
:100CAB000D2A908802E0F8C52D6830E00CC0E0A258
:100CBB006875F008120D2AD0E030E10CC0E0A26993
:100CCB0075F009120D2AD0E030E20CC0E0A26A7573
:100CDB00F00A120D2AD0E030E30CC0E0A26B75F0E5
:100CEB000B120D2AD0E030E40CC0E0A26C75F00CB6
:100CFB00120D2AD0E030E50CC0E0A26D75F00D129C
:100D0B000D2AD0E030E60CC0E0A26E75F00E120D8D
:100D1B002AD0E030E708A26F75F00F120D2A22924D
:100D2B000590257DE07003020E8CF54F754D007517
:100D3B004C26854D82854C83E0F9A3E0FAA3E0A312
:100D4B00A385824D85834C89828A83F545C0F075D6
:100D5B00F002A4F54B85F04AD0F0A3A31232D1FBDD
:100D6B00A31232D1FCA31232D1FDA31232D1FEA3B6
:100D7B001232D1FFEF547FB5F05EEB20E405200576
:100D8B00578003300552EE600CB407005007120E6B
:100D9B009040028043903000E5452582F582E0309B
:100DAB00E23030E02FE54B2400F582E54A3431F593
:100DBB00831213B9E582C39CE5839D5003020E8910
:100DCB00E545121E61758330854582E0D2E2F00263
:100DDB000E89D2E2F0020E89A31232D1FEA3123297
:100DEB00D1FFEF547FB5F02BEB20E50520052480D8
:100DFB000330051FEE600CB407005007120E904035
:100E0B00028010903000E5452582F582E0C2E2F0C9
:100E1B00020E89A31232D1FEA31232D1FFEF547FFF
:100E2B00B5F02BEB20E605200524800330051FEEE3
:100E3B00600CB407005007120E90400280109030E7
:100E4B0000E5452582F582E0D2E3F0020E89A3127C
:100E5B0032D1FEA31232D1FFEF547FB5F020EB203D
:100E6B00E7052005198003300514EE600CB407006C
:100E7B005007120E9040028005E545121E61D54FBA
:100E8B000122020D3DC082C083C0F0E5822407F52C
:100E9B0082E5833400F5831232D1F8A31232D15498
:100EAB001F240BF975A025E3F9EE30E708E8541F72
:100EBB00240BF8E2F8EE540F2323900EC973020FA4
:100ECB000900020F0D00020F1B00020F2900020F79
:100EDB003900020F4B00020F5B00020F0D00020FD7
:100EEB001B00020F2900020F3900020F4B00020FEB
:100EFB005B00020F0900020F0900020F0900C30279
:100F0B000F6DE988F0B5F004D3020F6DC3020F6DBE
:100F1B00E988F0B5F004C3020F6DD3020F6DE988B9
:100F2B00F0B5F0004004C3020F6DD3020F6DE988DA
:100F3B00F0B5F00280064004C3020F6DD3020F6DB3
:100F4B00E889F0B5F00040E2C3020F6DD3020F6DDC
:100F5B00E889F0B5F00280064004C3020F6DD3029E
:100F6B000F6DD0F0D083D08222200F030210A390FC
:100F7B00257EE070030210A3F54F754D00754C2ACA
:100F8B00854D82854C83E0F9A3E0FAA3E0A3A3850A
:100F9B00824D85834C89828A83F545C0F075F002BA
:100FAB00A4F54B85F04AD0F0A3A31232D1FBA312C8
:100FBB0032D1FCA31232D1FDA31232D1FEA31232D5
:100FCB00D1FFEE541FB40700404A1210A640028016
:100FDB0043903000E5452582F582E030E23030E089
:100FEB002FE54B2400F582E54A3431F5831213B912
:100FFB00E582C39CE5839D500302108FE545121ECD
:10100B0061758330854582E0D2E2F002108FD2E227
:10101B00F002108FA31232D1FEA31232D1FFEE5485
:10102B001FB4070040171210A6400280109030002A
:10103B00E5452582F582E0C2E2F002108FA3123261
:10104B00D1FEA31232D1FFEE541FB407004017128A
:10105B0010A640028010903000E5452582F582E015
:10106B00D2E3F002108FA31232D1FEA31232D1FFC2
:10107B00EE541FB40700400C1210A640028005E589
:10108B0045121E61D54F03021098020F8B7E2090E4
:10109B00252B7400F0A3DEFCC20F22C082C083C0DC
:1010AB00F0E5822407F582E5833400F5831232D113
:1010BB00F8A31232D1541FF990252B2582F582E02B
:1010CB00C2046002D204EE30E719E8541FF89025F1
:1010DB002B2582F582E06002D20475A025740B28C3
:1010EB00F8E2F830041275A025740B29F9E3F9EE38
:1010FB00540F2323900EC973C3D0F0D083D0822218
:10110B00854E4FE54E7003021364754B00754A30E4
:10111B00754D00754C2E900020E54E12136B858299
:10112B0047858346754300754231754520754400EC
:10113B00854B82854A83E020E2030212FA90001C61
:10114B001232D15401700890001B1232D1603285DB
:10115B0045828544831213A674152582F58274008B
:10116B003583F5831232D130E017C082C08320E182
:10117B0004740080027401903504F0D083D0828017
:10118B0011C082C0837400903504F0D083D08202EA
:10119B001273A31232D1F8A31232D1F9A31232D1A6
:1011AB00FA903502E0FB903501E0FC903500E0FD54
:1011BB00C3EB98F582EC99F5838542A0A843E582B1
:1011CB00F208E583F2ED9A30E70302126170719039
:1011DB003505854FF0C3E58225F0F582E5833400B4
:1011EB00F583E020E211E2701718E275F005B5F017
:1011FB0002800440028009903503E07003021289DB
:10120B00903504E070030212BA854782854683123B
:10121B0013A68582498583481213A6E58245836010
:10122B001F12137E600A854982854883A3A380E23F
:10123B00854D82854C83E549F0A3E548F00212ED1C
:10124B00903504E06069854D82854C83E549F0A3B8
:10125B00E548F00212ED8547828546831213A68579
:10126B0082498583480212ED85438285428312139E
:10127B00B9A38542A0A843E582F208E583F2854D28
:10128B0082854C831213B98582498583481213A634
:10129B00E5824583601912137E6047A3A3C20A122D
:1012AB00141920063D854982854883A3A380D890D5
:1012BB003504E0702D8547828546831213A68582FF
:1012CB00498583488542A0A8437400F208F2854BF8
:1012DB0082854A83E030E10510E3028002C2E2C25C
:1012EB00E4F0854D82854C83E549F0A3E548F08514
:1012FB004B82854A83E0F9903505854FF0C3E58233
:10130B0025F0F582E5833400F583E9F0D54F0280B3
:10131B0048854B82854A83A385824B85834A854DBD
:10132B0082854C83A3A385824D85834C854782851B
:10133B004683A3A385824785834685438285428363
:10134B00A3A3858243858342854582854483A3A3DA
:10135B0085824585834402113B9035037400F0224E
:10136B00C0F075F002A42582F582E5F03583F58394
:10137B00D0F022AD82AE831213A6AB82AC83854331
:10138B00828542831213B9E582C39BE5839C40049B
:10139B0074FF800274008D828E8322C0F01232D1D2
:1013AB00F5F0A31232D1F58385F082D0F022C0F094
:1013BB00E0F5F0A3E0F58385F082D0F022AA2412A9
:1013CB002D8922301347E550B4024214F5507800B2
:1013DB0075A02574FFF208E540F2087400F208E5E9
:1013EB002CF208E52DF208E52EF208E52FF2089015
:1013FB008000E0F208A3A3E0F208A3A3E0F208E464
:10140B00F208F29025007A007B2B122D9322C20654
:10141B00AD82AE837A001232E9FFA31232E9C21217
:10142B00B467004003D2122290391375F002A42541
:10143B0082F582E5F03583F583E493F5F0A3E4932D
:10144B0085F083F582E4731215FE0215F91216402E
:10145B000215F91216810215F91216C10215F912AD
:10146B0017070215F91217490215F9121758021529
:10147B00F91217970215F91217AF0215F91217C7C0
:10148B000215F91217F00215F91219470215F91284
:10149B0030580215F91219A50215F91219EC02159B
:1014AB00F9121B0F0215F9121C320215F9121C69E5
:1014BB000215F9121CB50215F9121D010215F912CC
:1014CB001D5B0215F9121C470215F9121DB5021509
:1014DB00F9121E1B0215F9121E340215F9121E4DBC
:1014EB000215F9121F820215F91220930215F91237
:1014FB0022BB0215F90215F9122CC10215F9122C97
:10150B00E10215F91223110215F912233F0215F905
:10151B001223E90215F912240D0215F912243902CE
:10152B0015F91224660215F91224970215F91224E3
:10153B00C60215F91224F90215F912252A0215F91A
:10154B001225640215F912259F0215F91225DE02E8
:10155B0015F912261B0215F912265C0215F9122633
:10156B009B0215F91226C20215F91226EB0215F988
:10157B001227170215F91227480215F912277B02B9
:10158B0015F91227B20215F91227E70215F91228DD
:10159B00200215F91228570215F91228960215F98F
:1015AB001228D70215F912291C0215F912295F020C
:1015BB0015F91229A60215F91229EB0215F9122AAF
:1015CB001A0215F912236D0215F91223A30215F94C
:1015DB00122A4B0215F9122AD40215F9122B0A0200
:1015EB0015F9122CAB0215F9122B490215F98D8244
:1015FB008E83228D828E83A3A31232E920E62912D9
:10160B0020F3B900104224F4F5F0902040E055F09F
:10161B00F05228801FB901104225F4F5F0902041BB
:10162B00E055F0F05229800C543F2474F5827583F9
:10163B002074FFF0228D828E83A3A31232E920E661
:10164B00281220F3F4B9000F5224F5F0902040E05B
:10165B0055F0F05228801EB9010F5225F5F090205D
:10166B0041E055F0F05229800C543F2474F58275FB
:10167B0083207400F0228D828E83A3A31232E9F8AB
:10168B00541F232400C81220F3FAA31232E975A0C9
:10169B0020F208F2EAB9000DF5F0902040E045F099
:1016AB00F042288010B9010DF5F0902041E045F093
:1016BB00F042298000228D828E83A3A31232E9F897
:1016CB00541F232400C81220F3FAA31232E975A089
:1016DB0020F208F2EAB9001042286224F4F5F090E7
:1016EB002040E055F0F08013B9011042296225F437
:1016FB00F5F0902041E055F0F08000228D828E8332
:10170B00A3A31232E920E6291220F3B900106224B8
:10171B00F4F5F0902040E055F0F05228801FB9010D
:10172B00106225F4F5F0902041E055F0F05229803D
:10173B000C543F2474F582758320E0F4F0228D82E3
:10174B008E83A3A31232E9FBA312219322902200D2
:10175B00E0F8A3E0F5F075A05D902100E0547FB4B4
:10176B000105790102177479009039E3E993600B55
:10177B00F20908E8B5F0F5D2068010902200E8C215
:10178B00ACF0200804D208D299D2AC228D828E8381
:10179B00A3A31232E9FAA31232E9FBA3122D936031
:1017AB0002D206228D828E83A3A31232E9FAA312F0
:1017BB0032E9FBA3122E0E6002D206228D828E839B
:1017CB00A3A31232E9FA7B01A31232E990250B2570
:1017DB0082F582A20AC0D0D20A122D93D0D0920ADF
:1017EB006002D206228D828E83A3A31232E9FAA362
:1017FB001232E9C0E0A31232E9FF540723239018F9
:10180B000D7302182C0002185E00021889000218D2
:10181B00AE0002182C0002182C0002182C00021823
:10182B002CD0E090250B2582F582E0780079007CA6
:10183B0000600F75F00A84A8F0600775F00A84A9A0
:10184B00F0FCE82430F8E92430F9EC2430FC7B037D
:10185B000218CCD0E090250B2582F582E0540F24A2
:10186B0030B43A0040022407F9E054F0C42430B4F9
:10187B003A0040022407FC78207B020218CCD0E00F
:10188B0090250B2582F582E054072430F8E054387C
:10189B000303032430F9E054C023232430FC7B03DF
:1018AB000218CCD0E090250B2582F5827B01A20A91
:1018BB00C0D0D20A122D93D0D0920A607ED206806D
:1018CB007AEF5438039018D4730218F300021927D7
:1018DB000002191800021901000218F3000218F394
:1018EB00000218F3000218F3BB0102802FBC302C4E
:1018FB00E9FCE8F9DBF2BC3023E9FCE8F97820BB22
:10190B00031ABC3017E9FCE8F97820800FBC300CC7
:10191B007C20BB0307B9300479208000902044EC75
:10192B00F0A3E9F0A3E8F0902044A20AC0D0D20AB9
:10193B00122D93D0D0920A6002D206228D828E8312
:10194B00A3A31232E9FAA31232E9F8A31232E9F98E
:10195B00A31232E990250B2582F582E0FB902044FF
:10196B007406F0A3E5404480F0FCA3E8F02CFCA344
:10197B007428F02CFCA3E9F02CFCA3EBF02CA303B4
:10198B00547FF09020447B07A20AC0D0D20A122DBC
:10199B0093D0D0920A6002D206228D828E8375D0AC
:1019AB0010A3A31232E9FBA3AD82AE83902100E515
:1019BB00822408F5827A01E0547FB40819A882A921
:1019CB00838D828E8375D000AA12AB13122D937563
:1019DB00D01088828983E5822408F5820ABA03D75E
:1019EB0022854B82854A83E0F98D828E83A3A312D5
:1019FB0032E9FA232323FC75A021F8E920E442E223
:101A0B00C2E7F2E408F208F2A31232E9FBA3122DAB
:101A1B009375A021ECF8E2D2E7F208080808081247
:101A2B0032E9F2A3081232E9F2200606A3081232B9
:101A3B00E9F2854B82854A83E0D2E4F0D206021BA1
:101A4B000E08A31232E924052582F582E43583F5CD
:101A5B00831232E9F5F0E2C395F0501E080808082E
:101A6B00E2F5F008E245F0602D18E2C39401F25064
:101A7B000408E214F2D206021B0EABF0A3EA245ABE
:101A8B00F5A078001232E9F5F0E2B5F009A308DB16
:101A9B00F3753803804A75A021EC2407F8E2600F38
:101AAB0014F28D828E83A3A3ECF8D206021A0A7568
:101ABB00373C30092B9000141232D1F8A31232D1DB
:101ACB00F5838882E5822AF582E43583F583123229
:101ADB00D1F8C3954E50097583308882E0D2E2F07D
:101AEB0075A021ECF8E2547FB403028003B4070421
:101AFB00C2E78002D2E7F2854B82854A83E0C2E4DB
:101B0B00F0C20622854B82854A83E0F98D828E8353
:101B1B00A3A31232E9FA232323FC75A021F8E920B1
:101B2B00E442E2C2E7F2E408F208F2A31232E9FB64
:101B3B00A3122E0E75A021ECF8E2D2E7F2080808EA
:101B4B0008081232E9F2A3081232E9F2200606A3C2
:101B5B00081232E9F2854B82854A83E0D2E4F0D257
:101B6B0006021C3108A31232E924052582F582E412
:101B7B003583F5831232E9F5F0E2C395F0501E0878
:101B8B00080808E2F5F008E245F0602D18E2C3946E
:101B9B0001F2500408E214F2D206021C31ABF0A39E
:101BAB00EA245AF5A078001232E9F5F0E2B5F00913
:101BBB00A308DBF3753803804A75A021EC2407F8E2
:101BCB00E2600F14F28D828E83A3A3ECF8D206028F
:101BDB001B2D75373C30092B9000141232D1F8A312
:101BEB001232D1F5838882E5822AF582E43583F5BA
:101BFB00831232D1F8C3954E50097583308882E039
:101C0B00D2E2F075A021ECF8E2547FB4030280031A
:101C1B00B40704C2E78002D2E7F2854B82854A8380
:101C2B00E0C2E4F0C206228D828E83A3A31232E9B6
:101C3B00547F232549F54950020548228D828E8316
:101C4B00A3A31232E9FAA31232E9F9EAC333FAE990
:101C5B0033F9EAC32549F549E93548F548228D8220
:101C6B008E83A3A31232E920E71810E60A1220F3A1
:101C7B00B900047824801E2474F875A020E2701A31
:101C8B008027547F1220F3B90004782C8007B90108
:101C9B0004782D8000567002800FA31232E9547F16
:101CAB00232549F54950020548228D828E83A3A333
:101CBB001232E920E71810E60A1220F3B900047873
:101CCB0024801E2474F875A020E2601A8027547FAC
:101CDB001220F3B90004782C8007B90104782D8009
:101CEB0000566002800FA31232E9547F232549F579
:101CFB004950020548228D828E83A3A31232E9201C
:101D0B00E71810E60A1220F3B900047824801E2489
:101D1B0074F875A020E2701A8035547F1220F3B945
:101D2B000004782C8007B90104782D8000567002CE
:101D3B00801DA31232E9FAA31232E9F9EAC333FA8E
:101D4B00E933F9EAC32549F549E9FA3548F548225B
:101D5B008D828E83A3A31232E920E71810E60A12B4
:101D6B0020F3B900047824801E2474F875A020E2B7
:101D7B00601A8035547F1220F3B90004782C800749
:101D8B00B90104782D8000566002801DA31232E940
:101D9B00FAA31232E9F9EAC333FAE933F9EAC325B4
:101DAB0049F549E9FA3548F548228D828E83A3A37C
:101DBB001232E9F8C3954E50567583308882E03065
:101DCB00E24A30E04AC004C005900020E812136BD1
:101DDB001213A6A3A3A31232D1FCA31232D1FDE896
:101DEB00C0F075F002A42400F582E5F03431F583E0
:101DFB00D0F01213B9E582C39CE5839DD005D004C6
:101E0B00400DE8121E617583308882E0D2E2F02229
:101E1B008D828E83A3A31232E9F8C3954E500975B8
:101E2B0083308882E0C2E2F0228D828E83A3A312DC
:101E3B0032E9F8C3954E50097583308882E0D2E3BE
:101E4B00F0228D828E83A3A31232E9F8C3954E50F4
:101E5B0004E8121E6122C000C003C004C0F0F89059
:101E6B000020E54E12136BE812136B1213A6AB8214
:101E7B00AC8375832EE875F002A4F582E5F035830B
:101E8B00F583EBF0A3ECF0758331E875F002A4F564
:101E9B0082E5F03583F583E4F0A3F0758330888217
:101EAB00E0C2E2C2E4F0C2E3D0F0D004D003D00031
:101EBB0022902200E0F875A05D902100E0547FB4E1
:101ECB0000047402F2089000021232D1A3F208123D
:101EDB0032D1F208902200E8C2ACF0200804D208FC
:101EEB00D299D2AC22C004C005C00675A025784B90
:101EFB00791075040075050075060CD5041DD50504
:101F0B001AD506177455C29BC299F59975040075BD
:101F1B000504D504FDD505FA02005B3098DDE59983
:101F2B00F2C298EA70011B1AEB7003EA601108D930
:101F3B00C1784B7910E21232BEA308D9F880AC7A83
:101F4B00007B20DAFEDBFC784B7910E21232BEA369
:101F5B0008D9F8902100E0547FB4011474AAC29BF5
:101F6B00C299F599750400750508D504FDD505FAD8
:101F7B00D006D005D00422C2AF8D828E83A3A312CC
:101F8B0032E9FAA31232E9FBE599C29874AAC29B13
:101F9B00C299F599900000121EF002005B8D828EA3
:101FAB0083A3A31232E9FAA31232E9FB90000212C7
:101FBB0032D1F8A31232D1C854F0241CC8500104FA
:101FCB00F5838882745A1232BEA374A51232BEA353
:101FDB00EA1232BEA3EB1232BEA3C000C0017500E1
:101FEB0000750100D500FDD501FAD001D000C2AFBC
:101FFB00E599C29874AAC29BC299F599121EF07406
:10200B00AAC29BC299F599750400750504D504FD08
:10201B00D505FA02005B2014FDC29BD214F5992260
:10202B009000021232D1F8A31232D1C854F0241C02
:10203B00C8500104F58388821232D1B45A18A31206
:10204B0032D1B4A511A31232D1FAA31232D1FBA310
:10205B00BA000CBB0009E4122021122021801AEADD
:10206B00122021EB1220211232D1A31220211ABAF5
:10207B00FF011BBA00F1BB00EE750400750504D51A
:10208B0004FDD505FA02005B9000021232D1FAA3CF
:10209B001232D1FB700CEA7009E4122021122021BC
:1020AB0080278A828B83A3A3AA82AB83EA12202187
:1020BB00EB1220219000001232D1A31220211ABA68
:1020CB00FF011BBA00F1BB00EE750400750504D5CA
:1020DB0004FDD505FA02005B8D828E83A3A3123219
:1020EB00E9C2136002D21322F95407C90303035444
:1020FB0003C0E07401B90002800323D9FDF9D0E0DD
:10210B00C922780079001232D128500109F8A3DCDA
:10211B0005BD00F28006BCFFED1D80EAE86A700782
:10212B00E96B7003E4800274FF2290000075A098A5
:10213B007802E230E70BA3E583B405F6C211022166
:10214B0092D2117A30122D277A30122D277A38122B
:10215B002D277A80122D277A06122D277A0C122D15
:10216B00277A01122D277A40122D277A5A122D46E3
:10217B007A40122D27122D68B45AC1903A14122DA1
:10218B00039039FA122D1522EB60627A80122D27FB
:10219B001232E9B404005029A3DB028050B40004CE
:1021AB007A808010B401047AC08009B402047A9456
:1021BB0080027AD41232E9A3543F2AFA122D2780D7
:1021CB002AB40C08A37A01122D27801FB40D03A388
:1021DB008014B40A03A3800EB40E2EDB11800EFA0A
:1021EB00122D46A380057AC0122D27DBA322A31242
:1021FB0032E914A3C082C08390250B2582F582E0BF
:10220B00D083D08212227780E2B40FD3DB0280DD41
:10221B00A31232E914A3C082C08390250B2582F54B
:10222B0082E0D083D08212223680C07C017A20C318
:10223B009464400C1C7A31C394644004C394640AC4
:10224B002464C0E0122D46D0E07A31C3940A4003D7
:10225B000A80F81A240AC0E0BA3005EC60027A2032
:10226B00122D46D0E02430FA122D46227C017A2022
:10227B00C39464400C1C7A31C394644004C39464CB
:10228B000A2464BA20028007C0E0122D46D0E07AFF
:10229B0031C3940A40030A80F81A240AC0E0BA300A
:1022AB0003EC7003122D46D0E02430FA122D462297
:1022BB008D828E83A3A31232E95403FB7005903AEF
:1022CB00478013B40105903A57800BB40205903A3E
:1022DB00678003903A777A01122D277C10E493FAEA
:1022EB00122D46A3DCF77C107AC0122D27EBC424E9
:1022FB0074F582758320E060047A3180027A3012A3
:10230B002D46A3DCF1228D828E83A3A31232E9FA30
:10231B00A31232E9FBEA4224F4F5F0902040E05599
:10232B00F0F05228EB4225F4F5F0902041E055F007
:10233B00F05229228D828E83A3A31232E9FAA312C3
:10234B0032E9FBEAF45224F5F0902040E055F0F02E
:10235B005228EBF45225F5F0902041E055F0F05265
:10236B0029228D828E83A3A31232E9FAA31232E9BA
:10237B00FBEA7011EBF524F4F5F0902040E055F0FA
:10238B00F052288012B4010FEBF525F4F5F09020F4
:10239B0041E055F0F05229228D828E83A3A3123295
:1023AB00E9FAA31232E9FBEA701875A025740B2B1E
:1023BB00F8E52CF275A025742B2BF874FFF2D20FD5
:1023CB00801BB4011875A025740B2BF8E52DF27545
:1023DB00A025742B2BF874FFF2D20F8000228D8274
:1023EB008E83A3A31232E9541FF9240BF8A31232E4
:1023FB00E975A025F275A025742B29F874FFF2D28C
:10240B000F228D828E83A3A31232E9541FF9240B62
:10241B00F875A025E2F5F0A31232E9B5F00FA3127F
:10242B0032E9547F232549F54950020548228D8214
:10243B008E83A3A31232E9541F240BF875A025E257
:10244B00F5F0A31232E9B5F002800FA31232E95472
:10245B007F232549F54950020548228D828E83A39F
:10246B00A31232E9541F240BF875A025E2F5F0A353
:10247B001232E9C5F0B5F0004002800FA31232E929
:10248B00547F232549F54950020548228D828E83BE
:10249B00A3A31232E9541F240BF875A025E2F5F023
:1024AB00A31232E9B5F0004002800FA31232E954B7
:1024BB007F232549F54950020548228D828E83A33F
:1024CB00A31232E9541F240BF875A025E2F5F0A3F3
:1024DB001232E9C5F0B5F00280044002800FA3125E
:1024EB0032E9547F232549F54950020548228D8254
:1024FB008E83A3A31232E9541F240BF875A025E297
:10250B00F5F0A31232E9B5F00280044002800FA36C
:10251B001232E9547F232549F54950020548228D93
:10252B00828E83A3A31232E9541FF9240BF875A0F2
:10253B0025E2F5F0A31232E9B5F01DA31232E9FA48
:10254B00A31232E9F9EAC333FAE933F9EAC32549AD
:10255B00F549E9FA3548F548228D828E83A3A312FB
:10256B0032E9541F240BF875A025E2F5F0A31232C3
:10257B00E9B5F002801DA31232E9FAA31232E9F990
:10258B00EAC333FAE933F9EAC32549F549E9FA35E0
:10259B0048F548228D828E83A3A31232E9541F245F
:1025AB000BF875A025E2F5F0A31232E9C5F0B5F0F2
:1025BB00004002801DA31232E9FAA31232E9F9EAB4
:1025CB00C333FAE933F9EAC32549F549E9FA354842
:1025DB00F548228D828E83A3A31232E9541F240B5C
:1025EB00F875A025E2F5F0A31232E9B5F000400230
:1025FB00801DA31232E9FAA31232E9F9EAC333FAC6
:10260B00E933F9EAC32549F549E9FA3548F5482292
:10261B008D828E83A3A31232E9541F240BF875A06D
:10262B0025E2F5F0A31232E9C5F0B5F002800440C3
:10263B0002801DA31232E9FAA31232E9F9EAC3337D
:10264B00FAE933F9EAC32549F549E9FA3548F5487A
:10265B00228D828E83A3A31232E9541F240BF875AB
:10266B00A025E2F5F0A31232E9B5F0028004400296
:10267B00801DA31232E9FAA31232E9F9EAC333FA45
:10268B00E933F9EAC32549F549E9FA3548F5482212
:10269B008D828E83A3A31232E9541FF9240BF87594
:1026AB00A025E2FAA31232E92AF275A025742B2990
:1026BB00F974FFF3D20F228D828E83A3A31232E91A
:1026CB00541FF9240BF875A025E2FAA31232E9CABC
:1026DB00C39AF275A025742B29F974FFF3D20F223C
:1026EB008D828E83A3A31232E9541FF5F0240BF8CD
:1026FB00A31232E9541F240BF975A025E3F275A040
:10270B0025742B25F0F874FFF2D20F228D828E8365
:10271B00A3A31232E9541F240BF875A025E2F5F0A0
:10272B00A31232E9541F240BF9E3B5F00FA31232B5
:10273B00E9547F232549F54950020548228D828EA5
:10274B0083A3A31232E9541F240BF875A025E2F5DD
:10275B00F0A31232E9541F240BF9E3B5F00280DC2D
:10276B00A31232E9547F232549F54950020548222B
:10277B008D828E83A3A31232E9541F240BF875A00C
:10278B0025E2F5F0A31232E9541F240BF9E3C5F04F
:10279B00B5F0004002800FA31232E9547F23254984
:1027AB00F54950020548228D828E83A3A31232E98C
:1027BB00541F240BF875A025E2F5F0A31232E9544F
:1027CB001F240BF9E3B5F0004002800FA31232E98E
:1027DB00547F232549F54950020548228D828E836B
:1027EB00A3A31232E9541F240BF875A025E2F5F0D0
:1027FB00A31232E9541F240BF9E3C5F0B5F00280A4
:10280B00044002800FA31232E9547F232549F54976
:10281B0050020548228D828E83A3A31232E9541FE6
:10282B00240BF875A025E2F5F0A31232E9541F240E
:10283B000BF9E3B5F00280044002800FA31232E9DA
:10284B00547F232549F54950020548228D828E83FA
:10285B00A3A31232E9541F240BF875A025E2F5F05F
:10286B00A31232E9541F240BF9E3B5F01DA3123266
:10287B00E9FAA31232E9F9EAC333FAE933F9EAC305
:10288B002549F549E9FA3548F548228D828E83A30F
:10289B00A31232E9541F240BF875A025E2F5F0A31F
:1028AB001232E9541F240BF9E3B5F00280DCA312BA
:1028BB0032E9FAA31232E9F9EAC333FAE933F9EA56
:1028CB00C32549F549E9FA3548F548228D828E83AF
:1028DB00A3A31232E9541F240BF875A025E2F5F0DF
:1028EB00A31232E9541F240BF9E3C5F0B5F00040F5
:1028FB0002801DA31232E9FAA31232E9F9EAC333BB
:10290B00FAE933F9EAC32549F549E9FA3548F548B7
:10291B00228D828E83A3A31232E9541F240BF875E8
:10292B00A025E2F5F0A31232E9541F240BF9E3B50D
:10293B00F0004002801DA31232E9FAA31232E9F92A
:10294B00EAC333FAE933F9EAC32549F549E9FA351C
:10295B0048F548228D828E83A3A31232E9541F249B
:10296B000BF875A025E2F5F0A31232E9541F240BE6
:10297B00F9E3C5F0B5F00280044002801DA31232CA
:10298B00E9FAA31232E9F9EAC333FAE933F9EAC3F4
:10299B002549F549E9FA3548F548228D828E83A3FE
:1029AB00A31232E9541F240BF875A025E2F5F0A30E
:1029BB001232E9541F240BF9E3B5F00280044002F4
:1029CB00801DA31232E9FAA31232E9F9EAC333FAF2
:1029DB00E933F9EAC32549F549E9FA3548F54822BF
:1029EB008D828E83A3A31232E9541FF5F0240BF8CA
:1029FB0075A025E2FAA31232E9541F240BF9E32A3E
:102A0B00F275A025742B25F0F874FFF2D20F228DEE
:102A1B00828E83A3A31232E9541FF5F0240BF875B1
:102A2B00A025E2FAA31232E9541F240BF9E3CAC31F
:102A3B009AF275A025742B25F0F874FFF2D20F22B1
:102A4B008D828E83A3A31232E9541FF9903A877AB1
:102A5B0001122D277C10E493FA122D46A3DCF77A92
:102A6B00C0122D279024007420F0A3F0A3F0A3F044
:102A7B00A3E904122C43EBB430027420F0A3EAF068
:102A8B00A37420F0A3743DF0A37420F0A375A025CC
:102A9B00E9240BF9E3122C43ECD204B43004C20446
:102AAB007420F0A3EBB430052004027420F0A3EAE9
:102ABB00F0A37420F0A3F0A3F0A3F07C10902400FB
:102ACB00E0FA122D46A3DCF8228D828E83A3A3128B
:102ADB0032E9541FF9FB75A025240BF9E3FA90009A
:102AEB001A1232D1C39401B408005012C423441FEC
:102AFB00F583EB44E0F582EA1232BE122CB6228D3E
:102B0B00828E83A3A31232E9541FF990001A12325A
:102B1B00D1C39401B408005024C423441FF583E9A6
:102B2B0044E0F5821232D1FA75A025740B29F8EA2C
:102B3B00F275A025742B29F874FFF2D20F22C0F086
:102B4B008D828E83A3A31232E975F03CA4FEAFF005
:102B5B00A31232E9C32EFEEF3400FFA31232E97544
:102B6B00F03CFB7C007D00C3EB2EFBEC3FFCED341B
:102B7B0000FD15F0E5F070EFA31232E9F879007A59
:102B8B00009000091232D1B4000575F0188013B40F
:102B9B00030575F019800BB4010575F01E800375E4
:102BAB00F01EC3E82BF8E93CF9EA3DFA15F0E5F025
:102BBB0070F09000091232D1B4013AEF700BEE6055
:102BCB0034B40A03022BD44018C3EE940AFEEF94DC
:102BDB0000FFC3E89412F8E99400F9EA9400FA8034
:102BEB00DAC3EE9401FEC3E89402F8E99400F9EA23
:102BFB009400FA80C6903500E0FD903501E0FC9022
:102C0B003502E0FBC3E89BFFE99C7014EA9D701052
:102C1B0090001B1232D1F5F0EFB5F00280084006A0
:102C2B009035037401F0903500EAF0903501E9F02E
:102C3B00903502E8F0D0F0227A007B007C00601621
:102C4B0075F00A84AAF0600E75F00A84ABF060068A
:102C5B0075F00A84ACF0EA2430FAEB2430FBEC2458
:102C6B0030FC229000001232D1FB9020001232D1A6
:102C7B00FDEBF41232BE122CB61232D1F4B5030EA8
:102C8B009000001232D1B503057A18022C9B7A08FA
:102C9B00902000ED1232BE122CB690257FEAF02266
:102CAB00122C6E90257FE0FAF599227C0075F0329C
:102CBB00DCFED5F0FB227A80122D277B2890258015
:102CCB00122D68F0A3DBF97AC0122D277B28122D69
:102CDB0068F0A3DBF9227A80122D277B28902580C0
:102CEB00E0FA122D46A3DBF87AC0122D277B28E0E1
:102CFB00FA122D46A3DBF8227A80122D277400934B
:102D0B006007FA122D46A380F4227AC0122D277485
:102D1B0000936007FA122D46A380F422C0F0301105
:102D2B001775F00075A0987802E230E70700D5F030
:102D3B00F3022D437800EAF2D0F022C0F030111AE2
:102D4B0075F00075A0987802E230E70700D5F0F334
:102D5B00022D6575A0987801EAF2D0F022C0F03010
:102D6B00111975F00075A0987802E230E70700D5CD
:102D7B00F0F3022D8675A0987803E2D0F02275A0AF
:102D8B00807800EAF4F22222AE82AF83902200EA2E
:102D9B002323232582F58274003583F583E0F8A382
:102DAB00E0F9EA245DF5A089F08E828F831232E977
:102DBB00F2A308E8B5F003022E07DBF1AE82AF8376
:102DCB00902200EA2323232582F58274003583F5B4
:102DDB0083E8BA000FC2ACF0200804D208D299D213
:102DEB00AC022E01D20BF0902064EA14540F258212
:102DFB00F582E0D2E7F0E48E828F832274FF8E821D
:102E0B008F8322AE82AF83902200EA232323258275
:102E1B00F58274003583F583E0F8A3E0F9EA245DCD
:102E2B00F5A089F08E828F831232E9B4F308DB1C94
:102E3B000BA3E8022EC1B4F408DB330BA3E8022E7C
:102E4B00C1B4F56EDB4A0BA3E8022EC1A31232E923
:102E5B00B4F303022EBD14A3C082C08390250B25AF
:102E6B0082F582E0D083D082122F17022EC1A312DB
:102E7B0032E9B4F403022EBD14A3C082C0839025A3
:102E8B000B2582F582E0D083D082122F68022EC1EF
:102E9B00A31232E9B4F503022EBD14A3C082C08382
:102EAB0090250B2582F582E0D083D082122F13025E
:102EBB002EC1122F13A3B5F006022F0C022E33DBFB
:102ECB00FBAE82AF83902200EA2323232582F58277
:102EDB0074003583F583E8BA000FC2ACF020080408
:102EEB00D208D299D2AC022F06D20BF0902064EA12
:102EFB0014540F2582F582E0D2E7F0E48E828F83A3
:102F0B002274FF8E828F8322F208E8227F017E20BB
:102F1B00C39464400C1F7E31C394644004C3946417
:102F2B000E2464BE2002800EC0E0EE122F13B5F00B
:102F3B0003022F67D0E07E31C3940A40030E80F862
:102F4B001E240AC0E0BE3003EF700AEE122F13B539
:102F5B00F003022F67D0E02430122F13227F017E63
:102F6B0030C39464400C1F7E31C394644004C394FB
:102F7B00640E2464C0E0EE122F13B5F003022FB5DC
:102F8B00D0E07E31C3940A40030E80F81E240AC0A1
:102F9B00E0BE3005EF60027E30EE122F13B5F0036A
:102FAB00022FB5D0E02430122F1322200B03023056
:102FBB00579000121232D1F5F0A31232D1F583855E
:102FCB00F082A3E5822411F582E5833400F583AE0C
:102FDB0082AF8390206475A0907A00C082C0838EEC
:102FEB00828F831232D154E0B4E007D083D08202B7
:102FFB00303FD083D082E030E73AC2E7F0EAC40337
:10300B002402F8C082C0838E828F831232D1B40A1D
:10301B00168FF07465F27FD7C2AFDFFE7475F27F47
:10302B0024DFFED2AFAFF0D083D08274A5F20808B4
:10303B00087406F2A3C082C0838E828F83A3AE82F4
:10304B00AF83D083D0820ABA0291C20B228D828EBB
:10305B0083A3A31232E914540FC40375A090240266
:10306B00F8A31232E9F9C2AF7465F274A5F27FDEF0
:10307B00E9DFFED9FCF97475F27F6FDFFED9FC74C2
:10308B00B5F2D2AF2290000A1232D16016758C00C5
:10309B00758A00D2A9D2AA7530FFF534853433D2A4
:1030AB00078039C2079000091232D1B40008753677
:1030BB006A753508801CB401087536877535E9804B
:1030CB0011B403087536707535088006753688752A
:1030DB00350885368C85358AC2AAD2A9D20222E55B
:1030EB004E700302318C854E4F7A007B007800794D
:1030FB002A7D0075F026754520754400854582852F
:10310B0044831213A6AE82AF8374052582F58274B5
:10311B00003583F5837C04C204C2051232D1A3604F
:10312B0002D2041232D1A3B4FF028002D205DCEB2F
:10313B0030041788828983EEF0A3EFF0A3E54EC32A
:10314B00954FF0A3A3A882A9830B3005198D828517
:10315B00F083EEF0A3EFF0A3E54EC3954FF0A3A3DE
:10316B00AD828583F00A854582854483A3A385823E
:10317B0045858344D54F8590257EEBF090257DEAE0
:10318B00F022C2A878087A007B029000121232D18A
:10319B00F5F0A31232D1F58385F082A31232D1F56B
:1031AB0023A3AE82AF83E5822410F582E58334003E
:1031BB00F5831232D1FD75A021BD00067400D2E754
:1031CB008055BD05067402D2E7804CBD060674021D
:1031DB00D2E78043BD0C067401D2E7803ABDE0060E
:1031EB007404D2E78031BD0D067405D2E78028BD8B
:1031FB0011067409D2E7801FBD0E067407C2E78063
:10320B0016BD0F067406D2E7800DBD10067408D2EA
:10321B00E780047403C2E7F2FCE82402F975A022EC
:10322B00ECF3BDE0030232A075A090EA2400F9098B
:10323B00097410F319197402A21EB392E0BD0002B7
:10324B008003BD0E0444188011A21BB392E4A21C90
:10325B0092E2A21D5004C2E4D2E3F37407301F02C2
:10326B00740FF3EA2401F99032B6E5235407FC936B
:10327B00F3EA2404F97488BC06028008BD050280B9
:10328B0003BD06027408F3EA2402F97401F3EA247D
:10329B0005F97404F38F838E82E82408F8EA240876
:1032AB00FADB0280030231A7D2A82244668899BBBD
:1032BB00CCCCBB30960FC083C0E0E58324A0F58354
:1032CB00D0E0F0D08322C083E58324A0209609C3ED
:1032DB009460F583E4938003F583E0D08322300D73
:1032EB0004E493801D300A03E08017C083E5832438
:1032FB00A0209609C39460F583E4938003F583E0E3
:10330B00D08322300706753000C28C32C0D0C0E0AB
:10331B00C083C08275D01030071C758C00758A0075
:10332B00D28CE40530B530037530FFD533058534C9
:10333B0033800302357CD55003755010E538B4004B
:10334B0004D2B480041538C2B4E537B40004D2B546
:10335B0080041537C2B5300005D54102C200E528FF
:10336B00700302346030401B902001E014F07013A6
:10337B00C240B220902040E030E008902000E0A353
:10338B00F0D24030411B902003E014F07013C24187
:10339B00B221902040E030E108902002E0A3F0D26F
:1033AB004130421B902005E014F07013C242B22250
:1033BB00902040E030E208902004E0A3F0D24230AD
:1033CB00431B902007E014F07013C243B2239020EC
:1033DB0040E030E308902006E0A3F0D24330441BDA
:1033EB00902009E014F07013C244B224902040E006
:1033FB0030E408902008E0A3F0D24430451B902025
:10340B000BE014F07013C245B225902040E030E57C
:10341B000890200AE0A3F0D24530461B90200DE027
:10342B0014F07013C246B226902040E030E60890AC
:10343B00200CE0A3F0D24630472290200FE014F08E
:10344B00701AC247B227902040E030E70F90200E51
:10345B00E0A3F0D247E529700302355730481B90A3
:10346B002011E014F07013C248B228902041E030D4
:10347B00E008902010E0A3F0D24830491B902013B5
:10348B00E014F07013C249B229902041E030E108FA
:10349B00902012E0A3F0D249304A1B902015E01483
:1034AB00F07013C24AB22A902041E030E20890201B
:1034BB0014E0A3F0D24A304B1B902017E014F070AD
:1034CB0013C24BB22B902041E030E308902016E062
:1034DB00A3F0D24B304C1B902019E014F07013C2A8
:1034EB004CB22C902041E030E408902018E0A3F07F
:1034FB00D24C304D1B90201BE014F07013C24DB218
:10350B002D902041E030E50890201AE0A3F0D24D39
:10351B00304E1B90201DE014F07013C24EB22E9053
:10352B002041E030E60890201CE0A3F0D24E304F53
:10353B001B90201FE014F07013C24FB22F9020414C
:10354B00E030E70890201EE0A3F0D24F30020FD2FC
:10355B0001853E83853F82A385833E85823F20077D
:10356B0010C28CE58A2535F58AE58C3536F58CD27B
:10357B008CD082D083D0E0D0D032C0D0C0E0C0831A
:10358B00C082C01F75D0182098113099030236598C
:10359B00D01FD082D083D0E0D0D032C298E5874400
:1035AB0040F587309F2AC29F902100E0547FB400E2
:1035BB00117401F0E58754BFF587759840D29C02D2
:1035CB0035DB7400F0E58754BFF5877598C0D29C46
:1035DB00E58754BFF587902100E0547FB4000302C8
:1035EB003602A3E0F58275835AE599F00582E582F0
:1035FB00902101F0023656902101E0F8A3E0F9A3E7
:10360B00E0FAA3E0FBE599FF309A1030E70DC29A80
:10361B007B01E8FA0AEA6970027B00EB6021758393
:10362B005A8A82EFF00582E5826970047B00800F75
:10363B00AA820B309A098882EB14F0EAF87B00908F
:10364B002101E8F0A3A3EAF0A3EBF0023592C299B3
:10365B00101403023663A192902200E0F8A3E0B5A8
:10366B00180CE4902203F0A3F0C208023592F890F4
:10367B002100E0547FB40031E8F8902204E070128E
:10368B0075835D8882E0902203F0902201E004F0C4
:10369B008011F8902203E014B5180CE4902203F08B
:1036AB00A314F0D29B8002C29B902201E075835D34
:1036BB00F582E0F5990582E582902201F0A3A3A3A0
:1036CB00E004F0023592C0D0C0E0C0F0C083C082ED
:1036DB0075D018753C02753D00753B00E53B90902D
:1036EB00052582F582E020E2030237BBC0E0902182
:1036FB0008E53B2582F582E0FCA385823A85833978
:10370B00547FB4000E909001E53B2582F582E0A238
:10371B00E5920C909003E53B2582F582E0F5F0EC09
:10372B0020E7030237B9547FB40003023759853AB7
:10373B0082853983E0F582E53D245BF583E5F0F086
:10374B000582E582853A82853983F00237B9853A5D
:10375B0082853983E0FCA3E0FDA3E0FEA3E0FFE557
:10376B00F0300C1030E70DC20C7F01ECFE0EEE6D4D
:10377B0070027F00EF60258E82E53D245BF583E5CB
:10378B00F0F00582E5826D70047F00800FAE820F32
:10379B00300C098C82EF14F0EEFC7F00902109E5D0
:1037AB003B2582F582ECF0A3A3EEF0A3EFF0D0E083
:1037BB0020E0030238F8902208E53D2323232582DD
:1037CB00F582E0FFA3E0B51F22A3A37400F0A3F0E2
:1037DB00909002E53B2582F58274B8F0909005E558
:1037EB003B2582F5827404F00238F8F5F085823AB5
:1037FB00858339A3E0547FB400028008B4070280AC
:10380B00030238D4C0E0A3E0FC600114FEA3E0FD8A
:10381B00D0E0B40705BC00538003BC001FE5F0F5F6
:10382B0082E53D245EF583E0FC0582E582853A82E4
:10383B00853983F0F5F0B51F070237D4EDB51E2B94
:10384B00909002E53B2582F5827415F0909000E58F
:10385B003B2582F582E0FEA3A37415F0909000E562
:10386B003B2582F582EE4404F08029909002E53BE3
:10387B002582F5827415F0909000E53B2582F58248
:10388B00E0FEA3A37415F0909000E53B2582F58232
:10389B00EE54FBF0E5F0F582E53D245EF583E0FEAA
:1038AB000582E582853A82853983F00DECB51D04DE
:1038BB007C007D00A3A3ECF0A3EDF0909003E53B1F
:1038CB002582F582EEF00238F8E5F0F582E53D242D
:1038DB005EF583E0F5F00582E582853A82853983D2
:1038EB00F0909003E53B2582F582E5F0F0053DE590
:1038FB003B2408F53BD53C0280030236E7D082D04F
:10390B0083D0F0D0E0D0D03215F915F914521458F9
:10391B00145E1464146A15001500150015031509BF
:10392B001470147C14B214B814BE14D014A61488DA
:10393B00148E149414A0149A14D614DC14E214E804
:10394B0014FA15001500150015CF15D5150F151503
:10395B0015E115E714AC1482151B15211527152D30
:10396B0015331539153F1569156F1575157B1581B0
:10397B001587158D1593159915C315C915DB14F4FA
:10398B0015ED1EBC1FA8202B14EE15F9147614C4CC
:10399B0014CA1545154B15511557155D1563159F14
:1039AB0015A515AB15B115B715BD150015001500EF
:1039BB001500150015001500150015001500150054
:1039CB00150015001500150015F3150015F915F95F
:1039DB0015F915F915F915F915496E7465724163E9
:1039EB0074697661746F722056362E35330D002054
:1039FB00496E746572416374697661746F72207677
:103A0B00362E3533202020200020416C636F726EE0
:103A1B00204D63427269646520002053686F7720E4
:103A2B00646174613A2062616420002053686F778F
:103A3B0020646174613A20206F6B200020466C611A
:103A4B00672042616E6B20232031202020466C6161
:103A5B00672042616E6B20232032202020466C6150
:103A6B00672042616E6B20232033202020466C613F
:103A7B00672042616E6B20232034202053746174C5
:103A8B0065205661726961626C65202357616974A8
:103A9B00696E6720666F7220202020202020202056
:103AAB00202020202020202020202020202020200B
:103ABB00202020200065787465726E616C2073790C
:103ACB006E632E2E2E202020202020202020202030
:103ADB00202020202020202020202020200045787E
:103AEB007465726E616C2073796E632020202020C8
:103AFB0020202020202020202020202020202020BB
:103B0B00202020202020007265636F76657265642B
:103B1B002E2020202020202020202020202020208C
:103B2B0020202020202020202020202020202000AA
:00000001FF
